******************************************************************************
               TMS320C6x Linker PC v7.3.4                      
******************************************************************************
>> Linked Wed Jan 08 18:17:57 2014

OUTPUT FILE NAME:   <mcasp_c674x_omapl137_evmOMAPL137.out>
ENTRY POINT SYMBOL: "_c_int00"  address: c00129e0


MEMORY CONFIGURATION

         name            origin    length      used     unused   attr    fill
----------------------  --------  ---------  --------  --------  ----  --------
  SHDSPL2ROM            11700000   00100000  00000000  00100000  RWIX
  SHDSPL2RAM            11800000   00040000  00000000  00040000  RWIX
  SHDSPL1PRAM           11e00000   00008000  00000000  00008000  RWIX
  SHDSPL1DRAM           11f00000   00008000  00000000  00008000  RWIX
  EMIFACS0              40000000   20000000  00000000  20000000  RWIX
  EMIFACS2              60000000   02000000  00000000  02000000  RWIX
  EMIFACS3              62000000   02000000  00000000  02000000  RWIX
  EMIFACS4              64000000   02000000  00000000  02000000  RWIX
  EMIFACS5              66000000   02000000  00000000  02000000  RWIX
  SHRAM                 80000000   00020000  00000000  00020000  RWIX
  DDR2                  c0000000   20000000  00012e4c  1ffed1b4  RWIX
  ARMROM                fffd0000   00010000  00000000  00010000  RWIX
  ARMRAM                ffff0000   00002000  00000000  00002000  RWIX


SECTION ALLOCATION MAP

 output                                  attributes/
section   page    origin      length       input sections
--------  ----  ----------  ----------   ----------------
.pinit     0    c0000000    00000000     UNINITIALIZED

.data      0    c0000000    00000000     UNINITIALIZED

.far       0    c0000000    0000be08     UNINITIALIZED
                  c0000000    0000bba8     omapl137_mcaspPlayBk.obj (.far)
                  c000bba8    00000240     system_config.lib : interrupt.obj (.far)
                  c000bde8    0000000c     omapl137_codecif.obj (.far)
                  c000bdf4    0000000c     rts6740.lib : exit.obj (.far)
                  c000be00    00000008                 : _lock.obj (.far)

.cinit     0    c000be08    000000e4     
                  c000be08    0000006c     omapl137_mcaspPlayBk.obj (.cinit)
                  c000be74    00000004     --HOLE-- [fill = 0]
                  c000be78    0000002c     rts6740.lib : exit.obj (.cinit)
                  c000bea4    00000004     --HOLE-- [fill = 0]
                  c000bea8    0000001c     omapl137_codecif.obj (.cinit)
                  c000bec4    00000004     --HOLE-- [fill = 0]
                  c000bec8    0000001c     rts6740.lib : _lock.obj (.cinit)
                  c000bee4    00000004     --HOLE-- [fill = 0]
                  c000bee8    00000004     (.pad.cinit) [fill = 0]

.const     0    c000bef0    0000005c     
                  c000bef0    00000040     omapl137_mcaspPlayBk.obj (.const)
                  c000bf30    0000000c     omapl137_mcaspPlayBk.obj (.const:_rxBufPtr)
                  c000bf3c    00000004     --HOLE-- [fill = 0]
                  c000bf40    0000000c     omapl137_mcaspPlayBk.obj (.const:_txBufPtr)

.bss       0    c000bf4c    00000024     UNINITIALIZED
                  c000bf4c    00000014     omapl137_mcaspPlayBk.obj (.bss)
                  c000bf60    0000000c     omapl137_codecif.obj (.bss)
                  c000bf6c    00000004     drivers.lib : edma.obj (.bss)

.text      0    c000c000    00006ae0     
                  c000c000    00001aa0     system_config.lib : interrupt.obj (.text:retain)
                  c000daa0    000017c0     drivers.lib : edma.obj (.text)
                  c000f260    00001260                 : mcasp.obj (.text)
                  c00104c0    00000900     omapl137_mcaspPlayBk.obj (.text)
                  c0010dc0    000005e0     system_config.lib : interrupt.obj (.text)
                  c00113a0    000004c0     drivers.lib : i2c.obj (.text)
                  c0011860    00000440     aic31.obj (.text)
                  c0011ca0    00000420     omapl137_codecif.obj (.text)
                  c00120c0    00000140     drivers.lib : psc.obj (.text)
                  c0012200    00000100     rts6740.lib : autoinit.obj (.text:__auto_init)
                  c0012300    000000e0                 : exit.obj (.text:_exit)
                  c00123e0    00000020                 : _lock.obj (.text:__nop)
                  c0012400    00000200     system_config.lib : intvecs.obj (.text)
                  c0012600    000000c0     rts6740.lib : divu.obj (.text:__divu)
                  c00126c0    000000a0                 : remu.obj (.text:__remu)
                  c0012760    000000a0                 : cpy_tbl.obj (.text:_copy_in)
                  c0012800    000000a0                 : memcpy64.obj (.text:_memcpy)
                  c00128a0    000000a0     platform.lib : i2c_omapl137.obj (.text)
                  c0012940    000000a0                  : mcasp_omapl137.obj (.text)
                  c00129e0    00000080     rts6740.lib : boot.obj (.text:_c_int00)
                  c0012a60    00000040                 : args_main.obj (.text:__args_main)
                  c0012aa0    00000020                 : exit.obj (.text:_abort)
                  c0012ac0    00000020     platform.lib : edma.obj (.text)

.stack     0    c0012ae0    00000400     UNINITIALIZED
                  c0012ae0    00000008     rts6740.lib : boot.obj (.stack)
                  c0012ae8    000003f8     --HOLE--


GLOBAL SYMBOLS: SORTED ALPHABETICALLY BY Name 

address    name
--------   ----
c000bf4c   $bss
c000bf4c   .bss
c0000000   .data
c000c000   .text
c0012aa0   C$$EXIT
c0011ba4   _AIC31ADCInit
c0011bf0   _AIC31DACInit
c0011880   _AIC31DataConfig
c0011860   _AIC31Reset
c001192c   _AIC31SampleRateConfig
c0012030   _CodecRegBitClr
c0011fb4   _CodecRegBitSet
c0011f6c   _CodecRegRead
c0011f28   _CodecRegWrite
c000de20   _EDMA3ChannelToParamMap
c000ebc8   _EDMA3ClearErrorBits
c000e1c4   _EDMA3ClrCCErr
c000e268   _EDMA3ClrEvt
c000e65c   _EDMA3ClrIntr
c000e0b4   _EDMA3ClrMissEvt
c000f068   _EDMA3ContextRestore
c000ee84   _EDMA3ContextSave
c000ed64   _EDMA3Deinit
c000dd5c   _EDMA3DisableChInShadowReg
c000e378   _EDMA3DisableDmaEvt
c000e5d4   _EDMA3DisableEvtIntr
c000e42c   _EDMA3DisableQdmaEvt
c000eb38   _EDMA3DisableTransfer
c000dc94   _EDMA3EnableChInShadowReg
c000e2f0   _EDMA3EnableDmaEvt
c000e54c   _EDMA3EnableEvtIntr
c000e3fc   _EDMA3EnableQdmaEvt
c000eaac   _EDMA3EnableTransfer
c000e504   _EDMA3ErrIntrHighStatusGet
c000ea0c   _EDMA3FreeChannel
c000e460   _EDMA3GetCCErrStatus
c000e4e0   _EDMA3GetErrIntrStatus
c000e484   _EDMA3GetIntrStatus
c000e6c4   _EDMA3GetPaRAM
c000daa0   _EDMA3Init
c000e4b0   _EDMA3IntrStatusHighGet
c000de44   _EDMA3MapChToEvtQ
c000df8c   _EDMA3MapQdmaChToPaRAM
c000dc80   _EDMA3PeripheralIdGet
c000e16c   _EDMA3QdmaClrMissEvt
c000e528   _EDMA3QdmaGetErrIntrStatus
c000e728   _EDMA3QdmaGetPaRAM
c000e8a4   _EDMA3QdmaGetPaRAMEntry
c000e7f8   _EDMA3QdmaSetPaRAM
c000e864   _EDMA3QdmaSetPaRAMEntry
c000e8ec   _EDMA3RequestChannel
c000e1e4   _EDMA3SetEvt
c000e78c   _EDMA3SetPaRAM
c000e078   _EDMA3SetQdmaTrigWord
c000df08   _EDMA3UnmapChToEvtQ
c0012ac0   _EDMAVersionGet
c0011218   _ExcCombineAdd
c0011260   _ExcCombineRemove
c00111f8   _ExcGlobalEnable
c0011cd8   _I2CCodecIfInit
c0011824   _I2CDMARxEventDisable
c00117d8   _I2CDMARxEventEnable
c0011800   _I2CDMATxEventDisable
c00117b4   _I2CDMATxEventEnable
c00117a0   _I2CDMATxRxEventDisable
c0011768   _I2CInterruptVectorGet
c00115c8   _I2CMasterBusBusy
c0011610   _I2CMasterControl
c00116e0   _I2CMasterDataGet
c00116b8   _I2CMasterDataPut
c0011478   _I2CMasterDisable
c0011440   _I2CMasterEnable
c0011690   _I2CMasterErr
c00113a0   _I2CMasterInitExpClk
c0011584   _I2CMasterIntClearEx
c00114e4   _I2CMasterIntDisableEx
c0011498   _I2CMasterIntEnableEx
c001152c   _I2CMasterIntStatus
c00115ec   _I2CMasterIsBusy
c00115b0   _I2CMasterSlaveAddrSet
c0011638   _I2CMasterStart
c0011658   _I2CMasterStop
c0011750   _I2COwnAddressSet
c00128a0   _I2CPinMuxSetup
c0011738   _I2CSetDataCount
c0011784   _I2CSlaveAddressGet
c0011720   _I2CSlaveDataGet
c00116f8   _I2CSlaveDataPut
c0011598   _I2CSlaveIntClearEx
c0011508   _I2CSlaveIntDisableEx
c00114c0   _I2CSlaveIntEnableEx
c0011548   _I2CSlaveIntStatus
c0011564   _I2CSlaveIntStatusEx
c0011678   _I2CStatusClear
c0010dc0   _IntDSPINTCInit
c0011170   _IntDisable
c0011140   _IntEnable
c0010f38   _IntEventClear
c0011074   _IntEventCombineAdd
c0010f70   _IntEventCombineInit
c0011118   _IntEventCombineRegister
c00110c8   _IntEventCombineRemove
c0010e7c   _IntEventMap
c0010f04   _IntEventSet
c00111cc   _IntGlobalDisable
c00111b8   _IntGlobalEnable
c00111e0   _IntGlobalRestore
c0010e30   _IntRegister
c00111a4   _IntReset
c0010e54   _IntUnRegister
c000f9e8   _McASPAMUTEINActivate
c000f938   _McASPAMuteDisable
c000f910   _McASPAMuteEnable
c0010294   _McASPContextRestore
c0010064   _McASPContextSave
c000ff80   _McASPDITChanStatRead
c000fec8   _McASPDITChanStatWrite
c000ffd4   _McASPDITChanUsrDataRead
c000ff24   _McASPDITChanUsrDataWrite
c000fea4   _McASPDITDisable
c000fe84   _McASPDITEnable
c000f8a8   _McASPPinDirInputSet
c000f878   _McASPPinDirOutputSet
c000f820   _McASPPinGPIOSet
c000f84c   _McASPPinMcASPSet
c0012940   _McASPPinMuxSetup
c000f2d8   _McASPReadFifoEnable
c000fe38   _McASPRxBufRead
c000f548   _McASPRxClkCfg
c000f9a4   _McASPRxClkCheckConfig
c000f638   _McASPRxClkPolaritySet
c000fc68   _McASPRxClkStart
c000fda8   _McASPRxEnable
c000f3e8   _McASPRxFmtI2SSet
c000f338   _McASPRxFmtMaskSet
c000f374   _McASPRxFmtSet
c000f470   _McASPRxFrameSyncCfg
c000f6c0   _McASPRxHFClkPolaritySet
c000fab4   _McASPRxIntDisable
c000fa60   _McASPRxIntEnable
c000f278   _McASPRxReset
c000fb54   _McASPRxSerActivate
c0010048   _McASPRxStatusGet
c000f8f4   _McASPRxTimeSlotSet
c000f7f0   _McASPSerializerInactivate
c000f798   _McASPSerializerRxSet
c000f744   _McASPSerializerTxSet
c000fe60   _McASPTxBufWrite
c000f49c   _McASPTxClkCfg
c000f960   _McASPTxClkCheckConfig
c000f5f4   _McASPTxClkPolaritySet
c000fbb0   _McASPTxClkStart
c000fcf8   _McASPTxEnable
c000f390   _McASPTxFmtI2SSet
c000f318   _McASPTxFmtMaskSet
c000f354   _McASPTxFmtSet
c000f440   _McASPTxFrameSyncCfg
c000f680   _McASPTxHFClkPolaritySet
c000fa8c   _McASPTxIntDisable
c000fa38   _McASPTxIntEnable
c000f260   _McASPTxReset
c000f724   _McASPTxRxClkSyncDisable
c000f704   _McASPTxRxClkSyncEnable
c000fae4   _McASPTxSerActivate
c001002c   _McASPTxStatusGet
c000f8d4   _McASPTxTimeSlotSet
c000f294   _McASPWriteFifoEnable
c00120c0   _PSCModuleControl
c0012ee0   __STACK_END
00000400   __STACK_SIZE
00000001   __TI_args_main
c000bdfc   ___TI_enable_exit_profile_output
ffffffff   ___TI_pprof_out_hndl
ffffffff   ___TI_prof_data_size
ffffffff   ___TI_prof_data_start
ffffffff   ___binit__
c000bf4c   ___bss__
ffffffff   ___c_args__
c000be08   ___cinit__
c0000000   ___data__
c0000000   ___edata__
c000bf70   ___end__
c0012ae0   ___etext__
ffffffff   ___pinit__
c000c000   ___text__
c0012a60   __args_main
c0012200   __auto_init
c0012600   __c6xabi_divu
c00126c0   __c6xabi_remu
c000bdf4   __cleanup_ptr
c0012600   __divu
c000bdf8   __dtors_ptr
c000be00   __lock
c00123e0   __nop
c00126c0   __remu
c0012ae0   __stack
c000be04   __unlock
c0012aa0   _abort
c000cff8   _c674x_mask_int10_isr
c000d1c0   _c674x_mask_int11_isr
c000d384   _c674x_mask_int12_isr
c000d548   _c674x_mask_int13_isr
c000d710   _c674x_mask_int14_isr
c000d8d8   _c674x_mask_int15_isr
c000c550   _c674x_mask_int4_isr
c000c718   _c674x_mask_int5_isr
c000c8e0   _c674x_mask_int6_isr
c000caa4   _c674x_mask_int7_isr
c000cc68   _c674x_mask_int8_isr
c000ce30   _c674x_mask_int9_isr
c000c000   _c674x_nmi_isr
c000c1c4   _c674x_rsvd_int2_isr
c000c388   _c674x_rsvd_int3_isr
c00129e0   _c_int00
c0012760   _copy_in
c000bf60   _dataIdx
c0012300   _exit
c0012400   _intcVectorTable
c0010ac0   _main
c0012800   _memcpy
c000bf6c   _regionId
c000bf68   _savedBase
c000bde8   _slaveData
c000bf64   _txCompFlag
ffffffff   binit
c000be08   cinit
c0000000   edata
c000bf70   end
c0012ae0   etext
ffffffff   pinit


GLOBAL SYMBOLS: SORTED BY Symbol Address 

address    name
--------   ----
00000001   __TI_args_main
00000400   __STACK_SIZE
c0000000   .data
c0000000   ___data__
c0000000   ___edata__
c0000000   edata
c000bde8   _slaveData
c000bdf4   __cleanup_ptr
c000bdf8   __dtors_ptr
c000bdfc   ___TI_enable_exit_profile_output
c000be00   __lock
c000be04   __unlock
c000be08   ___cinit__
c000be08   cinit
c000bf4c   $bss
c000bf4c   .bss
c000bf4c   ___bss__
c000bf60   _dataIdx
c000bf64   _txCompFlag
c000bf68   _savedBase
c000bf6c   _regionId
c000bf70   ___end__
c000bf70   end
c000c000   .text
c000c000   ___text__
c000c000   _c674x_nmi_isr
c000c1c4   _c674x_rsvd_int2_isr
c000c388   _c674x_rsvd_int3_isr
c000c550   _c674x_mask_int4_isr
c000c718   _c674x_mask_int5_isr
c000c8e0   _c674x_mask_int6_isr
c000caa4   _c674x_mask_int7_isr
c000cc68   _c674x_mask_int8_isr
c000ce30   _c674x_mask_int9_isr
c000cff8   _c674x_mask_int10_isr
c000d1c0   _c674x_mask_int11_isr
c000d384   _c674x_mask_int12_isr
c000d548   _c674x_mask_int13_isr
c000d710   _c674x_mask_int14_isr
c000d8d8   _c674x_mask_int15_isr
c000daa0   _EDMA3Init
c000dc80   _EDMA3PeripheralIdGet
c000dc94   _EDMA3EnableChInShadowReg
c000dd5c   _EDMA3DisableChInShadowReg
c000de20   _EDMA3ChannelToParamMap
c000de44   _EDMA3MapChToEvtQ
c000df08   _EDMA3UnmapChToEvtQ
c000df8c   _EDMA3MapQdmaChToPaRAM
c000e078   _EDMA3SetQdmaTrigWord
c000e0b4   _EDMA3ClrMissEvt
c000e16c   _EDMA3QdmaClrMissEvt
c000e1c4   _EDMA3ClrCCErr
c000e1e4   _EDMA3SetEvt
c000e268   _EDMA3ClrEvt
c000e2f0   _EDMA3EnableDmaEvt
c000e378   _EDMA3DisableDmaEvt
c000e3fc   _EDMA3EnableQdmaEvt
c000e42c   _EDMA3DisableQdmaEvt
c000e460   _EDMA3GetCCErrStatus
c000e484   _EDMA3GetIntrStatus
c000e4b0   _EDMA3IntrStatusHighGet
c000e4e0   _EDMA3GetErrIntrStatus
c000e504   _EDMA3ErrIntrHighStatusGet
c000e528   _EDMA3QdmaGetErrIntrStatus
c000e54c   _EDMA3EnableEvtIntr
c000e5d4   _EDMA3DisableEvtIntr
c000e65c   _EDMA3ClrIntr
c000e6c4   _EDMA3GetPaRAM
c000e728   _EDMA3QdmaGetPaRAM
c000e78c   _EDMA3SetPaRAM
c000e7f8   _EDMA3QdmaSetPaRAM
c000e864   _EDMA3QdmaSetPaRAMEntry
c000e8a4   _EDMA3QdmaGetPaRAMEntry
c000e8ec   _EDMA3RequestChannel
c000ea0c   _EDMA3FreeChannel
c000eaac   _EDMA3EnableTransfer
c000eb38   _EDMA3DisableTransfer
c000ebc8   _EDMA3ClearErrorBits
c000ed64   _EDMA3Deinit
c000ee84   _EDMA3ContextSave
c000f068   _EDMA3ContextRestore
c000f260   _McASPTxReset
c000f278   _McASPRxReset
c000f294   _McASPWriteFifoEnable
c000f2d8   _McASPReadFifoEnable
c000f318   _McASPTxFmtMaskSet
c000f338   _McASPRxFmtMaskSet
c000f354   _McASPTxFmtSet
c000f374   _McASPRxFmtSet
c000f390   _McASPTxFmtI2SSet
c000f3e8   _McASPRxFmtI2SSet
c000f440   _McASPTxFrameSyncCfg
c000f470   _McASPRxFrameSyncCfg
c000f49c   _McASPTxClkCfg
c000f548   _McASPRxClkCfg
c000f5f4   _McASPTxClkPolaritySet
c000f638   _McASPRxClkPolaritySet
c000f680   _McASPTxHFClkPolaritySet
c000f6c0   _McASPRxHFClkPolaritySet
c000f704   _McASPTxRxClkSyncEnable
c000f724   _McASPTxRxClkSyncDisable
c000f744   _McASPSerializerTxSet
c000f798   _McASPSerializerRxSet
c000f7f0   _McASPSerializerInactivate
c000f820   _McASPPinGPIOSet
c000f84c   _McASPPinMcASPSet
c000f878   _McASPPinDirOutputSet
c000f8a8   _McASPPinDirInputSet
c000f8d4   _McASPTxTimeSlotSet
c000f8f4   _McASPRxTimeSlotSet
c000f910   _McASPAMuteEnable
c000f938   _McASPAMuteDisable
c000f960   _McASPTxClkCheckConfig
c000f9a4   _McASPRxClkCheckConfig
c000f9e8   _McASPAMUTEINActivate
c000fa38   _McASPTxIntEnable
c000fa60   _McASPRxIntEnable
c000fa8c   _McASPTxIntDisable
c000fab4   _McASPRxIntDisable
c000fae4   _McASPTxSerActivate
c000fb54   _McASPRxSerActivate
c000fbb0   _McASPTxClkStart
c000fc68   _McASPRxClkStart
c000fcf8   _McASPTxEnable
c000fda8   _McASPRxEnable
c000fe38   _McASPRxBufRead
c000fe60   _McASPTxBufWrite
c000fe84   _McASPDITEnable
c000fea4   _McASPDITDisable
c000fec8   _McASPDITChanStatWrite
c000ff24   _McASPDITChanUsrDataWrite
c000ff80   _McASPDITChanStatRead
c000ffd4   _McASPDITChanUsrDataRead
c001002c   _McASPTxStatusGet
c0010048   _McASPRxStatusGet
c0010064   _McASPContextSave
c0010294   _McASPContextRestore
c0010ac0   _main
c0010dc0   _IntDSPINTCInit
c0010e30   _IntRegister
c0010e54   _IntUnRegister
c0010e7c   _IntEventMap
c0010f04   _IntEventSet
c0010f38   _IntEventClear
c0010f70   _IntEventCombineInit
c0011074   _IntEventCombineAdd
c00110c8   _IntEventCombineRemove
c0011118   _IntEventCombineRegister
c0011140   _IntEnable
c0011170   _IntDisable
c00111a4   _IntReset
c00111b8   _IntGlobalEnable
c00111cc   _IntGlobalDisable
c00111e0   _IntGlobalRestore
c00111f8   _ExcGlobalEnable
c0011218   _ExcCombineAdd
c0011260   _ExcCombineRemove
c00113a0   _I2CMasterInitExpClk
c0011440   _I2CMasterEnable
c0011478   _I2CMasterDisable
c0011498   _I2CMasterIntEnableEx
c00114c0   _I2CSlaveIntEnableEx
c00114e4   _I2CMasterIntDisableEx
c0011508   _I2CSlaveIntDisableEx
c001152c   _I2CMasterIntStatus
c0011548   _I2CSlaveIntStatus
c0011564   _I2CSlaveIntStatusEx
c0011584   _I2CMasterIntClearEx
c0011598   _I2CSlaveIntClearEx
c00115b0   _I2CMasterSlaveAddrSet
c00115c8   _I2CMasterBusBusy
c00115ec   _I2CMasterIsBusy
c0011610   _I2CMasterControl
c0011638   _I2CMasterStart
c0011658   _I2CMasterStop
c0011678   _I2CStatusClear
c0011690   _I2CMasterErr
c00116b8   _I2CMasterDataPut
c00116e0   _I2CMasterDataGet
c00116f8   _I2CSlaveDataPut
c0011720   _I2CSlaveDataGet
c0011738   _I2CSetDataCount
c0011750   _I2COwnAddressSet
c0011768   _I2CInterruptVectorGet
c0011784   _I2CSlaveAddressGet
c00117a0   _I2CDMATxRxEventDisable
c00117b4   _I2CDMATxEventEnable
c00117d8   _I2CDMARxEventEnable
c0011800   _I2CDMATxEventDisable
c0011824   _I2CDMARxEventDisable
c0011860   _AIC31Reset
c0011880   _AIC31DataConfig
c001192c   _AIC31SampleRateConfig
c0011ba4   _AIC31ADCInit
c0011bf0   _AIC31DACInit
c0011cd8   _I2CCodecIfInit
c0011f28   _CodecRegWrite
c0011f6c   _CodecRegRead
c0011fb4   _CodecRegBitSet
c0012030   _CodecRegBitClr
c00120c0   _PSCModuleControl
c0012200   __auto_init
c0012300   _exit
c00123e0   __nop
c0012400   _intcVectorTable
c0012600   __c6xabi_divu
c0012600   __divu
c00126c0   __c6xabi_remu
c00126c0   __remu
c0012760   _copy_in
c0012800   _memcpy
c00128a0   _I2CPinMuxSetup
c0012940   _McASPPinMuxSetup
c00129e0   _c_int00
c0012a60   __args_main
c0012aa0   C$$EXIT
c0012aa0   _abort
c0012ac0   _EDMAVersionGet
c0012ae0   ___etext__
c0012ae0   __stack
c0012ae0   etext
c0012ee0   __STACK_END
ffffffff   ___TI_pprof_out_hndl
ffffffff   ___TI_prof_data_size
ffffffff   ___TI_prof_data_start
ffffffff   ___binit__
ffffffff   ___c_args__
ffffffff   ___pinit__
ffffffff   binit
ffffffff   pinit

[230 symbols]
